:100000000C943F020C9477020C9477020C947702C4
:100010000C9477020C9477020C9477020C9477027C
:100020000C9477020C9477020C942E250C940026E5
:100030000C9422200C9477020C9477020C94770293
:100040000C9477020C9477020C9477020C9477024C
:100050000C9477020C94AA200C9477020C947702EB
:100060000C9477020C9477020C9477020C9477022C
:100070000C9477020C9477020C9477020C9477021C
:100080000C9477020C9477020C9477020C9477020C
:100090000C9477020C9477020C9477020C947702FC
:1000A0000C9477020C9477020C9477023205320597
:1000B0005E055E05C605E405FC06FC06EF05880640
:1000C000990699066D2694268C2794268C27E0267F
:1000D00003278C275A27692707634236B79BD8A77F
:1000E0001A39685618AEBAAB558C1D3CB7CC57635D
:1000F000BD6DEDFD753EF6177231BF000000803F0B
:1001000005A84CCDB2D44EB93836A9020C50B991DD
:100110008688083CA6AAAA2ABE000000803F2E00BE
:100120001E001F002000210022000000000023000C
:1001300024002500260027002D002B0014001A00A3
:10014000080015001700000000001C0018000C003B
:1001500012001300310029000400160007000900F6
:100160000A00500052000B000D000E000F0033007B
:100170003400E1001D001B000600190005005100BD
:100180004F0011001000360037003800E500E00095
:10019000E300E200350001512A004C0028002C0049
:1001A0002F003000E600E700E400C65CC75CC85CD6
:1001B000C95CCA5CCB5C00000000010001000100CA
:1001C00001000100005C01004200430044004500C2
:1001D000460000000000010035002F003000010043
:1001E000010039003E003F00400041004900C45C6E
:1001F000C35C5000510052004F000100010001009B
:100200003A003B003C003D004800CE5CC55C4A0023
:100210004E004B004D0001000100010001000100F3
:1002200001000100010001000100010001000100C6
:1002300001000100010000047F3F1F64321464329A
:1002400014783C1E1E140A05FFAA7F5540000101C8
:100250000101010101010102020202020202020285
:100260000303030303030303040404040404040555
:100270000505050506060606060707070707080819
:100280000808090909090A0A0A0B0B0B0C0C0C0DCA
:100290000D0D0E0E0E0F0F0F101011111112121363
:1002A000131414151516161717181819191A1A1BDE
:1002B0001B1C1D1D1E1E1F2020212222232424253D
:1002C0002626272829292A2B2C2D2D2E2F30313276
:1002D00032333435363738393A3B3C3D3E3F404186
:1002E00042434445464748494A4C4D4E4F5051536E
:1002F00054555658595A5B5D5E5F61626465666825
:10030000696B6C6D6F7072737577787A7B7D7E80A8
:1003100082838587888A8C8E8F91939596989A9CF4
:100320009EA0A2A3A5A7A9ABADAFB1B3B5B7BABC08
:10033000BEC0C2C4C6C9CBCDCFD1D4D6D8DBDDDFD9
:10034000E2E4E7E9EBEEF0F3F5F8FAFDFF0E035314
:100350000070006500650064006F00000012034338
:10036000006F007A0079004B00650079007300008F
:10037000000403090409023B00020100A0FA090479
:1003800000000103010100092111010001224000C8
:1003900007058103080001090401000103000000B2
:1003A000092111010001227B0007058203200001C1
:1003B0001201000200000008EDFE9211030001028C
:1003C000000105010902A10185020901A100050939
:1003D00019012908150025019508750181020501FB
:1003E000093009311581257F950275088106093884
:1003F0001581257F950175088106050C0A380215BF
:1004000081257F950175088106C0C005010980A17D
:1004100001850319012AB700150126B7009501755A
:10042000108100C0050C0901A101850419012AA051
:1004300002150126A002950175108100C005010971
:1004400006A101050719E029E715002501950875A2
:100450000181029501750881010507190029FF1521
:100460000026FF0095067508810005081901290579
:10047000950575019102950175039101C000112444
:100480001FBECFEFDAE0DEBFCDBF04B603FE18C05B
:100490008091E5029091E602A091E702B091E80216
:1004A0008730904BA740B04B59F41092E502109260
:1004B000E6021092E7021092E802E0E0F8E3099504
:1004C00011E0A0E0B1E0E0E1F8E502C005900D9296
:1004D000A63CB107D9F722E0A6ECB1E001C01D921D
:1004E000A53EB207E1F70E94EB120C94062C0C9487
:1004F000000081E0089581E008950C947B02089546
:100500000C947F021F93CF93DF9300D000D01F92F3
:10051000CDB7DEB749835A836B833091C901898196
:100520009A81311114C0662359F0222349F00E94A8
:100530003909182F682F89819A810E94E20803C027
:100540000E940D09182F69817A81812F04C00E94B1
:10055000390969817A810F900F900F900F900F9059
:10056000DF91CF911F910C946D10FC01262F4081DB
:1005700051816281738184810C94820281E00895AB
:10058000CF93DF93EC0160E00E94B502BE01DF91E2
:10059000CF910C9480020C949C110C9498110895A6
:1005A0000E948C070E94CF022FEF84E39CE0215031
:1005B00080409040E1F700C000000C94D0200F93E1
:1005C0001F93CF93DF938C0161E00E94B502EC0191
:1005D000B8010E947D02882309F444C0B801CE010D
:1005E0000E94ED1E8823F1F1B801CE010E94011D89
:1005F0008823C1F1B801CE010E94491E882391F1E0
:10060000B801CE010E94071C882361F1F8018281A4
:10061000882309F1CB358DE5D807C1F050F4C11519
:10062000FCE5DF0781F0CF3DDC45A9F40E946A0EAE
:1006300019C0CC35EDE5DE0761F0CD35DD4559F467
:100640000E94B30D08C00E94D0020CC00E94BC0DD5
:1006500002C00E94BF0DC801DF91CF911F910F9181
:100660000C94790280E0DF91CF911F910F91089552
:100670000E9404200E9455030C94841A0E9458037F
:100680000E94501B0C940A2008950C94440381E0AE
:1006900008950C9447030895CF93C82F0E944503F3
:1006A0008C2F0E944903CF91089580E00C944C0355
:1006B0000E94491F0C944C030E94491F9091C8014D
:1006C000891721F08093C8010C944C030895CF93AF
:1006D000DF93CDB7DEB72B970FB6F894DEBF0FBE12
:1006E000CDBF4F83588769877A878B8761110E94B6
:1006F000FF0C9E012F5F3F4F86E0F90111928A9512
:10070000E9F785E0FE013796D90101900D928A95AF
:10071000E1F789819A814C815D81452B31F09F3FC2
:1007200031F491E08F3F19F403C091E001C090E0F3
:1007300090FF09C049815A816B817C818D819E81A6
:100740000E94200C05C0C9010E94BE028111F2CF97
:100750002B960FB6F894DEBF0FBECDBFDF91CF91C1
:100760000895FC01808191810E947B090895CF93B7
:10077000882309F4A4C0C82F8238C1F40E94491FFD
:1007800081FD9DC069E380910201909103010E9467
:10079000DC1F0E94210D2FEF81EE94E0215080405C
:1007A0009040E1F700C0000069E319C0833801F50B
:1007B0000E94491F80FD83C063E5809102019091F2
:1007C00003010E94DC1F0E94210D2FEF81EE94E0B7
:1007D000215080409040E1F700C0000063E5809127
:1007E0000201909103010E94DE1FCF910C94210D14
:1007F0008438C1F40E94491F82FD61C067E4809182
:100800000201909103010E94DC1F0E94210D2FEF35
:1008100081EE94E0215080409040E1F700C000005C
:1008200067E4DDCF8CEF8C0F813AD0F46C2F809190
:100830000201909103010E94A61F882349F06C2FAA
:1008400080910201909103010E94DE1F0E94210D00
:100850006C2F80910201909103010E94DC1FC5CF93
:1008600080E28C0F883048F4C77081E001C0880FA7
:10087000CA95EAF70E94E20CB8CFEBE5EC0FE33043
:1008800040F4F0E0E65AFE4F808190E0CF910C9466
:100890006E1FE8E5EC0FE73150F4F0E0EE0FFF1FBC
:1008A000E45DFE4F80819181CF910C94841FCD3EF9
:1008B00030F08C2F0E947013CF910C944214CF9182
:1008C0000895882309F464C0823879F40E94491F8E
:1008D00081FF5EC069E380910201909103010E9453
:1008E000DC1F0E94210D69E310C08338B1F40E941F
:1008F000491F80FF4DC063E5809102019091030183
:100900000E94DC1F0E94210D63E5809102019091FD
:1009100003010E94DE1F0C94210D843879F40E949B
:10092000491F82FF35C067E4809102019091030165
:100930000E94DC1F0E94210D67E4E7CF9CEF980F17
:10094000913A10F4682FE1CF90E2980F983050F46C
:10095000877091E001C0990F8A95EAF7892F0E946C
:10096000E80CD9CF9BE5980F933020F480E090E01D
:100970000C946E1F98E5980F973120F480E090E07A
:100980000C94841F8D3E20F00E94CB130C944214D3
:1009900008951F93CF93DF93182FEB010E94B703A5
:1009A000209741F08FE99FE00197F1F700C0000028
:1009B0002197F6CF812FDF91CF911F910C94610485
:1009C000893319F060E070E002C060E570E00C94DB
:1009D000C904882321F00E94E20C0C94210D089593
:1009E000882321F00E94E80C0C94210D0895CF92E9
:1009F000DF92EF92FF920F931F93CF93DF937C01CF
:100A0000D62FC72FFC011281058102950F700E941D
:100A1000D80C8823B9F01123A9F08C2F807F803463
:100A200021F080E28D0F883068F08091960282FD7F
:100A300009C082E00E94810D0E94D80C91E0D82E5E
:100A4000D92601C0D12CCC2EC2948FE0C8228C2D87
:100A500090E08C30910508F0CFC1FC01EA5AFF4FBD
:100A60000C94612B8C2F807FCF70882311F0C2955E
:100A7000C07F112399F0CC2309F4AAC180E28D0F25
:100A8000883010F0D11104C08C2F0E94E20C03C0FA
:100A90008C2F0E94F20C0E94210D9AC18D2F0E9472
:100AA0006104CC2309F4A8C180E28D0F883038F1AD
:100AB000DD2329F18C2F0E94F80C24C08C2F807F1D
:100AC000CF70803211F0C295C07FDD2319F0D13094
:100AD000A1F13DC08091960282FF17C0112349F019
:100AE000CC2329F08C2F0E94E20C0E94210D80E083
:100AF00070C180E00E946104CC2309F47DC18C2F79
:100B00000E94E80C0E94210D77C1112371F000238F
:100B100041F0013031F40E94020D8C2B0E940A0D2D
:100B20006BC10E94020D8C2B1DC0002319F00130F7
:100B300009F462C10E94170D25C0112321F006306F
:100B400008F05AC10EC0053008F056C11BC0112371
:100B500061F0002331F0F701858180FF39C18F708A
:100B600085838C2F0E94E90447C1002359F0D933B3
:100B700009F03FC1FFEF07EE13E0F15000401040D5
:100B8000E1F735C18C2F0E94F00436C18C2F869579
:100B90008695837019F0813061F02EC1112321F008
:100BA0008D2F9C2F937002C080E090E00E946E1FFA
:100BB0002BC1112321F08D2F9C2F937002C080E058
:100BC00090E00E94841F20C18D2F112319F00E94F4
:100BD000701302C00E94CB130E94421415C18C2FC7
:100BE000837009F047C011110BC12D2F2295269556
:100BF0002770220F220F6D2F6F70862F90E0A0E0DC
:100C0000B0E0022E04C0880F991FAA1FBB1F0A94D0
:100C1000D2F7D4FF10C04FE050E060E070E004C0B5
:100C2000440F551F661F771F2A95D2F740955095A0
:100C30006095709503C040E050E0BA01C695C69536
:100C4000C3708A019B01082B192B2A2B3B2BC9014E
:100C5000B801C23049F058F4C13019F00E94F807C9
:100C6000CFC00E94E607CCC00E940A08C9C00E94FB
:100C7000E407C6C0112319F08C2F817001C086953E
:100C8000882309F4BDC02D2F229526952770220FA9
:100C9000220F6D2F6F70862F90E0A0E0B0E0022E43
:100CA00004C0880F991FAA1FBB1F0A94D2F7D4FF54
:100CB00010C04FE050E060E070E004C0440F551FEA
:100CC000661F771F2A95D2F74095509560957095CD
:100CD00003C040E050E0BA01C695C695C3708A01D2
:100CE0009B01082B192B2A2B3B2BC901B801C230C1
:100CF00049F058F4C13019F00E94BD0881C00E942B
:100D0000AB087EC00E94CF087BC00E941E0878C03E
:100D1000CF70112339F08C2F0E9444088D2F0E9430
:100D2000E9046EC08D2F0E94F0048C2F0E9465088C
:100D300067C0D23F21F128F4D03F41F0D13FC1F04C
:100D400043C0D33F19F1D43F79F03EC0112341F0A5
:100D5000053008F051C08C2F8F710E948A084CC05A
:100D6000063008F049C0F7CF8091960282FF18C084
:100D7000112339F08C2F8F710E9444083DC011233C
:100D8000C9F38C2F8F710E94650836C0112329F09A
:100D90008C2F8F710E942F082FC00E942A082CC010
:100DA000112349F0CF718C2F0E94440863E08C2FEF
:100DB0000E94660D21C081E00E94810D0230E0F0AA
:100DC00082E00E94810D18C0112331F0002391F2BE
:100DD0008D2F0E94B70310C0002399F2D93349F434
:100DE0001FEF27EE33E0115020403040E1F700C004
:100DF00000008D2F0E94610488EF8C0D843020F458
:100E00000E94491F0E944C03DD20C9F00E94D40CAF
:100E100080FD15C0F70112820E94CE0C0E9444088A
:100E2000C7010E9440070E94CE0CDF91CF911F9115
:100E30000F91FF90EF90DF90CF900C946508DF91B9
:100E4000CF911F910F91FF90EF90DF90CF90089579
:100E50000F931F93CF93DF93EC01688179818A818F
:100E60000E9486098C010E94E1080E94D207B80105
:100E7000CE010E94F704DF91CF911F910F91089549
:100E8000CF93DF93EC01988189812B813C81232BC7
:100E900031F08F3F31F481E09F3F19F403C081E0CE
:100EA00001C080E080FD1DC0CE010E94DF028111E3
:100EB00010C00E94D80C8823A1F08A81882389F071
:100EC0008091960282FD0DC082E0DF91CF910C945B
:100ED000810DCE010E942807CE01DF91CF910C94A5
:100EE000C002DF91CF91089580E090E00E946E1FD4
:100EF00080E090E00E94841F0E94FF0C0E94210D60
:100F00000E9473150C944214809102019091030188
:100F10000E94E01F0C9474070E94EF0C0C9484074D
:100F200092959F70963079F010F4925001C09A50CB
:100F3000923068F4803F69F018F4883E40F409C0AC
:100F4000843F29F406C0883E20F0813F11F080E004
:100F5000089581E00895FC01808191810E947B09C0
:100F60000E9490070895CF93DF9300D000D01F9286
:100F7000CDB7DEB70F900F900F900F900F90DF91CD
:100F8000CF910895CF93DF9300D000D000D0CDB79C
:100F9000DEB726960FB6F894DEBF0FBECDBFDF9149
:100FA000CF910895089508950C94D3070C94D40715
:100FB0000E94D6076093FB017093FC018093FD01B2
:100FC0009093FE010C9474070C94D8070F931F9311
:100FD0000091FB011091FC012091FD013091FE0177
:100FE000602B712B822B932B1F910F910C94D807A0
:100FF0000F931F930091FB011091FC012091FD01C3
:101000003091FE0160237123822393231F910F915E
:101010000C94D8070F931F930091FB011091FC01D2
:101020002091FD013091FE016027712782279327CF
:101030001F910F910C94D8070C94D3070E941C08A1
:101040006093F7017093F8018093F9019093FA018E
:101050000C94740760E070E0CB010C941E080F93B1
:101060001F9341E050E060E070E08A019B0104C002
:10107000000F111F221F331F8A95D2F7C901B80133
:101080001F910F910C941E080F931F9341E050E0A5
:1010900060E070E004C0440F551F661F771F8A95FB
:1010A000D2F78091F7019091F801A091F901B091E8
:1010B000FA018A019B01082B192B2A2B3B2BC90112
:1010C000B8011F910F910C941E080F931F9341E0DC
:1010D00050E060E070E004C0440F551F661F771FAA
:1010E0008A95D2F740955095609570958091F7015B
:1010F0009091F801A091F901B091FA018A019B0148
:10110000082319232A233B23C901B8011F910F91FA
:101110000C941E080F931F9341E050E060E070E0D4
:1011200004C0440F551F661F771F8A95D2F7809120
:10113000F7019091F801A091F901B091FA018A01AB
:101140009B01082719272A273B27C901B8011F91AE
:101150000F910C941E080F931F930091F7011091AB
:10116000F8012091F9013091FA01602B712B822B4B
:10117000932B1F910F910C941E080F931F930091B6
:10118000F7011091F8012091F9013091FA016023E3
:101190007123822393231F910F910C941E080F93A8
:1011A0001F930091F7011091F8012091F9013091FE
:1011B000FA0160277127822793271F910F910C94C2
:1011C0001E0808952EE0929F800D1124E82FE695C9
:1011D000E695E695877051E001C0550F8A95EAF7CC
:1011E00085E0E89FF0011124E653FE4F20E030E057
:1011F00070E04081CB01022E02C0969587950A943B
:10120000E2F78170819584278523842781932F5F5E
:101210003F4F2530310569F708952EE0929F800DEC
:101220001124682F669566956695982F977085E0CE
:10123000689FB001112440E050E080E0FB01E40F22
:10124000F51FE653FE4F208130E0092E02C036958F
:1012500027950A94E2F721703327042E01C0220F4C
:101260000A94EAF7822B4F5F5F4F4530510531F703
:101270000895BF92CF92DF92EF92FF920F931F9348
:10128000CF93DF938C01C090F701D090F801E090EC
:10129000F901F090FA018091FB019091FC01A0917D
:1012A000FD01B091FE01C82AD92AEA2AFB2ACFE122
:1012B000D0E0D701C6010C2E04C0B695A79597952E
:1012C00087950A94D2F780FD04C0219790F7B12C3E
:1012D00007C0BC2EB8018C2F0E9480100197A9F383
:1012E0008B2DDF91CF911F910F91FF90EF90DF90A9
:1012F000CF90BF900895CF93DF93EC010E943909FE
:10130000BE010E948010DF91CF9108951F93CF936B
:10131000DF93EB019091C901992321F0CB010E9449
:101320007B0913C0882349F0CB010E943909182F8B
:10133000682FCE010E94E20804C0CB010E940D0973
:10134000182FBE01812F0E948010DF91CF911F9135
:1013500008951F93CF93DF93C091FF0116E0809112
:101360000002C81799F0D0E01C9FF0011D9FF00DFE
:101370001124EF5FFD4F408151816281738184812F
:1013800095810E94C2072196C770E9CFDF91CF9166
:101390001F910895409131025091320260913302C1
:1013A0007091340280913502909136020C94C207FC
:1013B000EF92FF920F931F93CF93DF9380913602AA
:1013C00082958F7009F065C080913302882309F4FB
:1013D00060C08091FF01F0900002109131020091F5
:1013E0003202609134027091350291E01F3F09F0A2
:1013F00090E0C0910001D0910101292F96E0E92EE3
:101400008F1509F446C06115710521F00F3F21F0D9
:1014100030E003C031E001C0322F90E030FD36C033
:10142000E89EF001E99EF00D1124DF01AF5FBD4F92
:1014300011963C911197301329C03C91311326C06D
:1014400012963C911297311121C013964D915C91E7
:101450001497461B570B4C175D07C0F4809136025A
:101460008F70806180933602EA5FFD4F80818F70BC
:101470008061808381E392E00E944007DF91CF91F9
:101480001F910F91FF90EF900C94A909019687701E
:10149000B7CFDF91CF911F910F91FF90EF900895FB
:1014A0009F92AF92BF92CF92DF92EF92FF920F93F3
:1014B0001F93CF93DF93CDB7DEB761970FB6F89444
:1014C000DEBF0FBECDBF8C0185E0F801DE011D96A9
:1014D00001900D928A95E1F7D8011296EC909091C7
:1014E0003102E0913202209134023091350221150F
:1014F000310531F0EF3F31F481E09F3F19F403C033
:1015000081E001C080E0B82FB1709B2E80FD47C103
:10151000D8014C9111965C9111971396AD90BC90A7
:10152000149781E3C82E82E0D82EF0903302B501E3
:10153000621B730B2091000130910101FF2009F41F
:10154000D9C0809136026217730708F095C0282F22
:10155000207F09F052C05E1313C0491311C0FE2C46
:10156000E1100EC08F708061809336020E94CA091C
:10157000C6010E94400780913602F80185834DC163
:10158000AB2831F05F3F31F481E04F3F19F403C0E5
:1015900081E001C080E080FD03C081E08E2502C0B3
:1015A00080E090E0F82FF170FF2E80FF1CC080914A
:1015B000FF012091000236E0821709F40BC190E090
:1015C000389FF001399FF00D1124EF5FFD4F6181CD
:1015D000561306C06081461303C06281E61203C041
:1015E00001968770E9CFFE2CEE2009F416C1809198
:1015F000360281608093360254C05E1306C04913E0
:1016000004C0E11002C0F80199C0C8010E94AB07F4
:10161000882361F1EE2051F120913602822F8295CC
:101620008F7090E0029774F08091310290913202B5
:1016300098878F831986BB86AA862C87CE0107964A
:101640000E94400786E0F801A1E3B2E001900D920C
:101650008A95E1F70E94D8090E94CA090AC05E175C
:1016600011F1C8010E94AB0781112CC0C8010E9472
:101670004007FF24F394D1C0282F207F81F77A2DD3
:10168000B98AA88A6E2D89890E94B30781E392E006
:101690000E94400786E0D6011D928A95E9F70E94D4
:1016A000CA09F12CBAC04913DCCFE110DACFF80136
:1016B0008583C8010E94400786E0D6011D928A9565
:1016C000E9F7ABC0EE2091F220913602822F82958D
:1016D0008F7090E002970CF4B5CF80913102909119
:1016E00032029A8389831B82BD82AC822E83CE0113
:1016F0000196A6CF6217730708F044C0FE2CEE20B7
:1017000009F4B4CF5E1330C049132EC020913602C5
:1017100020FD21C0822F82958F70482F50E0411507
:101720005105C9F0F80125834F30510541F08F5F15
:10173000982F9295907F822F8F70892B8583C80177
:101740000E94400786E0F801A1E3B2E001900D920B
:101750008A95E1F73CC086E0F801A1E3B2E0019090
:101760000D928A95E1F759C0C8010E94AB0781111B
:1017700069CF80913602816080933602C8010E9451
:1017800040074BC07A2DB98AA88A6E2D89890E949C
:10179000B30786E0D6011D928A95E9F718C0EE20BE
:1017A00009F464CFC8010E94AB07F82E882309F41E
:1017B0005DCF86E0F801A1E3B2E001900D928A9539
:1017C000E1F781E392E00E94B1030E94D8090E94F0
:1017D000CA0923C04D875E878D859E850E947B093F
:1017E000292F22952F70223028F49F7039F0811113
:1017F00005C00BC0243028F49F7049F4805E883007
:1018000020F0C8010E9440079F2CF92C06C0D80187
:1018100015969C91907F91F7F8CF8F2D61960FB61A
:10182000F894DEBF0FBECDBFDF91CF911F910F9116
:10183000FF90EF90DF90CF90BF90AF909F90089572
:101840001F93CF93DF93CDB7DEB72C970FB6F894E5
:10185000DEBF0FBECDBF4F83588769877A878B87DE
:101860009C87CE0107960E94500A8823D1F09F8161
:1018700088852A853B85232B31F08F3F31F481E029
:101880009F3F19F403C081E001C080E080FD47C0A4
:101890004F81588569857A858B859C850E94C20712
:1018A0003EC086E0FE013796DE01119601900D9252
:1018B0008A95E1F7FF81E8856A857B856115710569
:1018C00031F0EF3F31F481E0FF3F19F403C081E0D4
:1018D00001C080E080FD23C02091000230E0C901FA
:1018E0000196877099274091FF0150E08417950772
:1018F000F1F1F983EA837D836C8396E0929FD001B6
:10190000939FB00D1124AF5FBD4FFE013196019042
:101910000D929A95E1F7809300020E94A90916E0C2
:101920008091FF0190910002891771F1189FC00109
:1019300011248F5F9D4F0E94500A882329F1E09166
:10194000FF011E9FF0011124EF5FFD4F4081518187
:1019500062817381848195810E94C2078091FF0119
:1019600090E00196877099278093FF01D9CF0E945C
:101970008C07109200021092FF01E1E3F2E086E092
:10198000DF011D928A95E9F72C960FB6F894DEBF19
:101990000FBECDBFDF91CF911F91089580913F027F
:1019A000859585958595089580913F028770089566
:1019B00090913F02977081E009F480E00895809152
:1019C0004A02089590914A02892B80934A02089511
:1019D000809590914A02892380934A02089510923B
:1019E0004A02089590914902892B809349020895F3
:1019F000809590914902892380934902089510921D
:101A00004902089580914002089508950C94050DAF
:101A10000C94060D9091960292FD08C090914002A0
:101A2000981721F0809340020C94080D089580913E
:101A30004002882329F01092400280E00C94080DA7
:101A40000895CF93DF93E0910201F091030180911B
:101A50004A028083E0910201F0910301908180911C
:101A60004902892B808380914002882381F0E09194
:101A70000201F09103019081892B80838091020102
:101A8000909103010E949A1F81110E94170DC0912D
:101A90000201D091030148E050E067E372E0CE011B
:101AA0000E94B12B892B69F088E0FE01A7E3B2E028
:101AB00001900D928A95E1F7CE01DF91CF910C94C0
:101AC000551FDF91CF9108950C94050D90919602CA
:101AD00092FD10C098E0899F90011124262B20933D
:101AE0003F020E94440880913F0285958595859527
:101AF0000C94640D0C94440810923F0280E00C9406
:101B0000640D20913F028095822380933F02982F9D
:101B1000977099F430E0482F082E000C550B2417CD
:101B2000350759F09091960292FD07C085958595ED
:101B300085950E9465080C947C0D089590919602FD
:101B400092FB222720F9281769F080FB92F99093E5
:101B5000960280919502909196020E94E60D82E095
:101B60000C94810D08958091960282FB882780F95C
:101B700091E089270C949E0D81E00C949E0D80E0ED
:101B80000C949E0D80E090E00E94CC2B21E0893ED9
:101B90009E4F09F020E0822F089582E090E00C949F
:101BA000BE2B83E090E00C94BE2BCF9384E090E0BA
:101BB0000E94BE2BC82F82E290E00E94BE2B2C2FE9
:101BC00030E0A901582BCA01CF910895CF93C92FB6
:101BD000682F84E090E00E94D22B6C2F82E290E08C
:101BE000CF910C94D22BAB01BC018FE090E00C9410
:101BF000E42BAB01BC0183E190E00C94E42B60E0AA
:101C000070E0CB010C94F90D60E070E0CB010E9414
:101C1000F30D0C94FF0D69EE7EEF80E090E00E94E2
:101C2000F02B60E082E090E00E94D22B60E083E045
:101C300090E00E94D22B1092FB011092FC011092B6
:101C4000FD011092FE0160E084E090E00E94D22B42
:101C500060E082E290E00E94D22B60E085E090E0BC
:101C60000E94D22B60E086E090E00E94D22B6FEFC2
:101C700087E090E00E94D22B40E050E0BA0188E07B
:101C800090E00E94E42B60E08DE090E00E94D22B77
:101C900040E050E0BA0188E190E00E94E42B60E06F
:101CA00087E190E00E94D22B40E050E0BA018CE145
:101CB00090E00E94E42B60E070E080E290E00E94FF
:101CC000F02B40E050E0BA0188E190E00E94E42B64
:101CD0000C94040E0C940B0E682F8EE090E00C9484
:101CE000D22B0E948F206093590270935A028093E6
:101CF0005B0290935C02609355027093560280934E
:101D0000570290935802089585B7806885BF85B7BC
:101D1000806885BF089581E008950C948B0E089526
:101D20000C948F0E0C948F0E0C94920E0C948F0EBC
:101D30000C94960E0C948F0E0E94840E8CE591E10B
:101D40000E943F1F0E949A0E0C94980E0E94900EC3
:101D50000C948F0E0E945F110C944B030E947A200A
:101D60000E9444120E94AA0E0E94151B0C94940E0D
:101D70005F926F927F928F929F92AF92BF92CF921B
:101D8000DF92EF92FF920F931F93CF93DF93CDB724
:101D9000DEB72A970FB6F894DEBF0FBECDBF0E9404
:101DA0005912C82E81110E94710E3BE4832E32E03D
:101DB000932E00E010E0502E802F0E9483115C01D2
:101DC000F401619071904F016826792661147104C5
:101DD000B1F40F5F1F4F0530110569F78FEF89834D
:101DE0008A831B820E9483208160782F9D838C834D
:101DF00049815A816B818D810E9467033AC080912D
:101E00005D0281FD0E948C11D12CEE24E394F12C13
:101E1000C3018E219F21892B29F10E948D0E8823D9
:101E2000A9F0DE825F82AE20BF2081E0AB2809F4FA
:101E300080E088870E9483208160782F9A87898735
:101E40004E815F8168858A850E946703000F111F9C
:101E5000F801E55BFD4F80819181E826F926F1824A
:101E6000E08207C0D394EE0CFF1CFEE0DF12D0CF5F
:101E7000B0CF81E0C11001C080E02A960FB6F8947F
:101E8000DEBF0FBECDBFDF91CF911F910F91FF90AD
:101E9000EF90DF90CF90BF90AF909F908F907F900A
:101EA0006F905F9008950E94B80E0E94591B0E9487
:101EB00060140C945C03CF93DF930E948510EC01B7
:101EC000811521E5920708F045C0811530E593079B
:101ED00008F094C0883E910528F5803E910508F0F1
:101EE000F8C0883A910570F4853A910508F07CC0F5
:101EF0008130910509F475C008F4E8C0049708F032
:101F0000E8C0E4C08F3B910508F0E0C0C85AD0E0BB
:101F1000CC0FDD1FC35ADE4F0990D881C02DCE01F2
:101F20009464D8C0811540E2940758F4811551E0BB
:101F3000950708F0CEC08D3E910508F4C7C09065A6
:101F4000C9C0C11580E4D80708F4C0C0DF70CE0155
:101F5000906AC0C0811525E59207A8F4811534E583
:101F6000930708F095C0811543E5940708F07BC0FE
:101F7000811552E5950708F061C0D82FCC27CE0116
:101F8000816F906AA7C0C11589E5D807A0F4C11573
:101F900028E5D20708F082C0C11536E5D30708F05E
:101FA00095C08C2F0E9419118F7190E0D82FCC27EB
:101FB000CE0190628FC0C1154AE5D40708F474C001
:101FC000CE0190568115904208F080C08D2F8F7100
:101FD0000E941911DD27D0628F71AE01582BCA0102
:101FE00079C081E090E076C0C55AD0E0C557DE4F99
:101FF0008881C82FD0E0CE0190646CC074E09695C3
:1020000087957A95E1F7282F23703C2F337081E074
:1020100090E002C0880F991F3A95E2F79C68AC01E6
:10202000522B9A019C2F9F709695969550E2959F02
:10203000E0011124C9018C2B9D2B4CC08370992782
:1020400021E030E002C0220F331F8A95E2F79C2F77
:102050009695969580E2989FE0011124C22BD32B90
:10206000CE019C6837C08370992721E030E002C020
:10207000220F331F8A95E2F79C2F9695969540E2A2
:10208000949FE0011124C22BD32BCE019A6822C069
:10209000D82FCC27CE01846F906A1CC0DC2FCC27B0
:1020A000CE01806F906A16C08C2F8F700E9419111C
:1020B00094E0D695C7959A95E1F7CF70D0E0DC2FE4
:1020C000CC27D0699E01282BC90104C080E090E094
:1020D00001C0CE01DF91CF91089526E4829FC00117
:1020E0001124FC012EE0729FE00DF11D1124E60F7A
:1020F000F11DEE0FFF1FE25EFE4F85919491089552
:102100000E946D100E945B0F08958238910569F15D
:10211000B0F48133910509F46DC048F4893291051A
:1021200009F463C08A32910509F469C008958533C2
:10213000910509F455C089339105B9F00895833E9E
:10214000910569F138F4803E9105B1F0823E910528
:1021500009F10895863E9105A9F1873E9105B9F1EF
:10216000843E910509F064C023C02091950220FDB2
:102170004FC021FD4DC008958091950280FD44C05F
:102180008091960280FF44C08091950284FD42C0F8
:1021900083EE4DC08091950282FF38C0F5CF8091CB
:1021A000950282FD33C08091960280FD31C0ECCF54
:1021B0008091960281FF32C08091950284FD2AC0F1
:1021C00087EE35C08091950283FF26C0F5CF8091C0
:1021D000950283FD21C08091960281FD1FC0ECCF46
:1021E0008091950285FD1CC01DC08091950285FDE2
:1021F00019C016C08091950286FD16C017C0809147
:10220000950286FD13C010C089E311C082EE0FC095
:1022100080EE0DC080E00BC086EE09C084EE07C0E2
:1022200089E205C085E303C08AE201C081E390E052
:1022300008959091950292FF0DC0282F28712830A3
:1022400019F4877F846006C0282F2471243011F48C
:102250008B7F886093FF0DC0282F2871283119F4D7
:10226000877E846106C0282F2471243111F48B7E6F
:1022700088612091960220FF0DC0382F38713830C8
:1022800019F4877F816006C0382F3171313011F425
:102290008E7F886021FF0DC0282F2871283119F406
:1022A000877E816106C0282F2171213111F48E7E35
:1022B000886194FD877E089580E0089508950E94C6
:1022C000C20D811102C00E946A0E0E94CD0D809342
:1022D0005D020E94D50D90939602809395020E9414
:1022E0005E110E94D10D682F70E080E090E00E94A6
:1022F000E4076091F7017091F8018091F9019091E4
:10230000FA010C941C08E82FF0E0EE0FFF1FEF55C8
:10231000FD4F808191810895089580EA8A95F1F7B3
:10232000089500C008950C948D1108950C94951192
:102330000C9496110C9495110C949A11F894E82F22
:10234000E295EF70F0E031A1282F2F7081E090E04E
:1023500001C0880F2A95EAF7982F9095932391A3AF
:1023600092A1892B82A3789408950F931F93CF9302
:10237000DF93CCE9D1E089918F3F11F00E949E114B
:1023800081E0C13AD807B9F7CEE8D1E00CE911E015
:1023900089918F3F11F00E949E110C171D07C1F704
:1023A000DF91CF911F910F910895BF92CF92DF924D
:1023B000EF92FF920F931F93CF93DF938C01C62F61
:1023C000D0E0CE0184569E4F6C01FC0190819F3F6E
:1023D00009F450C0B62EF894E92FE295EF70F0E0C2
:1023E00081A19F7021E030E001C0220F9A95EAF7A9
:1023F000822B81A382A12095282322A378940E9476
:102400009111EEE8F1E04CE951E021E030E0E12CFF
:10241000F12C61916F3F89F0A62FA295AF70B0E0CB
:1024200090968C9190E06F7002C0959587956A9513
:10243000E2F780FD02C0C90102C080E090E0E82A16
:10244000F92A220F331F4E175F0719F7F601808113
:102450008F3F11F00E949E1161E0E114F10409F434
:1024600060E08B2D0E949311CC0FDD1FC00FD11F98
:10247000F982E882DF91CF911F910F91FF90EF9049
:10248000DF90CF90BF9008950E94B5118AE0E1EAF5
:10249000F2E0DF01982F1D929A95E9F7E7E9F2E063
:1024A000DF011D928A95E9F785E00E94A4120C9441
:1024B000CB02FF920F931F93CF93DF93CDB7DEB77D
:1024C0002A970FB6F894DEBF0FBECDBF8E010F5F07
:1024D0001F4F8AE0F80111928A95E9F7F12C6F2DD0
:1024E000C8010E94D511F394F5E0FF12F8CF4AE03D
:1024F00050E0B80187E992E00E94B12BFF24F394E9
:10250000009709F4F12C892B41F08AE0F801A7E942
:10251000B2E001900D928A95E1F72F2D45E061EA36
:1025200072E087E992E00E94A5120E94CD028F2DF1
:102530002A960FB6F894DEBF0FBECDBFDF91CF91C4
:102540001F910F91FF9008950895FF920F931F938D
:10255000CF93DF93F82E092F162FD72FC42F2223C6
:1025600049F081E0809360020E94832090935F0293
:1025700080935E02809160028823D9F080915E0290
:1025800090915F020E949B20059798F0EF2DF02F0D
:10259000A12FBD2F80E090E04C2F50E084179507CD
:1025A00034F4219131912D933D930196F7CF109200
:1025B0006002DF91CF911F910F91FF9008950E94CB
:1025C00086220E94AE0E0C9492220E9496220E94B5
:1025D000530F0C94B0220E9421200E946D220E9471
:1025E0009C0E0E94DF120E94E5120E94A60EFBCFF5
:1025F0008091670280FF06C06091090170E0660F5C
:10260000771F26C081FF04C06091090184E005C0E6
:1026100082FF07C06091090188E0689FB001112422
:1026200017C0909166029923D1F060910801961726
:1026300088F72091090188E0289F90011124929F3A
:10264000A001939F500D112470E0CA010E942B2B12
:102650006038710540F46115710519F406C068E031
:1026600070E0862F08958FE7089581E008958091A6
:10267000670280FF08C06091050170E0759567955D
:102680007595679521C081FF06C06091050170E0D6
:102690007595679519C082FF04C06091050170E0CF
:1026A00010C090916502992399F0609104019617EA
:1026B000A0F780910501899FC001112470E00E945C
:1026C0002B2B6038710540F46115710519F406C0B3
:1026D00061E070E0862F08958FE7089581E0089506
:1026E0008D3E21F40E94F812819504C08E3E29F49B
:1026F0000E94F81280936B0208958F3E21F40E948D
:10270000F812819504C0803F29F40E94F81280934A
:102710006A020895893F19F40E94371305C08A3F61
:1027200031F40E943713819580936C0208958B3F9A
:1027300021F40E943713819504C08C3F29F40E9434
:10274000371380936D0208959FE0980F983078F4C6
:1027500021E030E0A90102C0440F551F9A95E2F72D
:10276000CA0190916902892B8093690208958D3F77
:1027700021F48091670281600BC08E3F21F480912B
:102780006702826005C08F3F29F4809167028460F0
:102790008093670208958D3E39F490916B0297FF04
:1027A00035C010926B0259C08E3E29F490916B0295
:1027B0001916BCF32BC090916A028F3E29F497FF43
:1027C00025C010926A0249C0803F19F41916CCF353
:1027D0001DC090916C02893F29F41916BCF4109227
:1027E0006C023BC08A3F19F497FF10C0F8CF8B3FB3
:1027F00039F490916D0297FF09C010926D022DC0BF
:102800008C3F21F490916D021916BCF39FE0980F54
:10281000983080F421E030E0A90102C0440F551F38
:102820009A95E2F7CA018095909169028923809375
:10283000690213C08D3F21F4809167028E7F0BC027
:102840008E3F21F4809167028D7F05C08F3F29F470
:10285000809167028B7F8093670280916A02811169
:1028600006C080916B02811102C0109266028091B5
:102870006C02811106C080916D02811102C010921C
:10288000650208950E94832020916A02211104C0EC
:1028900020916B02222321F09093640280936302C3
:1028A00020916C02211104C020916D02222321F09D
:1028B000909362028093610288E692E00C94601F1C
:1028C000EF92FF920F931F93CF93DF9300D000D02E
:1028D00000D0CDB7DEB786E0E8E6F2E0DE01119683
:1028E00001900D928A95E1F7E0906A02F0906B02F8
:1028F00000916C0210916D0210926A0210926B02AC
:1029000010926C0210926D02E11003C0FF2009F4D6
:102910005DC080916302909164020E949B20AC0193
:1029200090916602992339F020910A0130E0241732
:10293000350758F04BC020910B018AE0289F900189
:1029400011242417350718F041C09F3F19F09F5FED
:1029500090936602EE2061F00E94F8121E1414F0AB
:102960009FEF01C091E0989F902D112490936A02EF
:10297000FF2061F00E94F8121F1414F09FEF01C0B5
:1029800091E0989F902D112490936B0230916A02F0
:102990003323E1F020916B022223C1F045EB340395
:1029A000C0011124992319F090936A0203C081E0B9
:1029B00080936A0235EB2303C0011124992319F097
:1029C00090936B0203C081E080936B02011103C0FE
:1029D000112309F45DC080916102909162020E940E
:1029E0009B20AC0190916502992339F0209106015A
:1029F00030E02417350758F04BC0209107018AE0DA
:102A0000289F900111242417350718F041C09F3FDB
:102A100019F09F5F90936502002361F00E943713C5
:102A2000101614F09FEF01C091E0989F902D112493
:102A300090936C02112361F00E943713111614F069
:102A40009FEF01C091E0989F902D112490936D020B
:102A500030916C023323E1F020916D022223C1F00A
:102A600045EB3403C0011124992319F090936C02B3
:102A700003C081E080936C0235EB2303C001112475
:102A8000992319F090936D0203C081E080936D0249
:102A900080916A0281110BC080916B02811107C085
:102AA00080916C02811103C080916D0281110E949E
:102AB0004214EB82FC820D831E8386E0FE01319678
:102AC000A8E6B2E001900D928A95E1F726960FB63E
:102AD000F894DEBF0FBECDBFDF91CF911F910F9154
:102AE000FF90EF900895E8E6F2E086E0DF011D92A6
:102AF0008A95E9F7109266021092650210926702B9
:102B00000895EF92FF920F931F93CF93DF938B0162
:102B1000682F11110AC0442329F0E82FF0E0E35B8D
:102B2000FD4F6491762F862F75C0212F30E0E82F5E
:102B3000F0E0442321F0E35BFD4FE491F0E046E058
:102B4000049FC0011124CFEFD0E0BE010E94172BDB
:102B50004BEA4603C001479F900D1124800F911D41
:102B6000800F911D982F990F890FAE01421B530BB7
:102B70004E9FD0014F9FB00D5E9FB00D11249B2F33
:102B8000189FA0011124452F55278E01041B150BFA
:102B90000E9FA0010F9F500D1E9F500D11247E010E
:102BA000E81AF108E29E8001E39E100DF29E100DDE
:102BB0001124212F3327C21BD30BCE9F9001CF9F0F
:102BC000300DDE9F300D112462307105A9F048F4FC
:102BD0006115710569F061307105C9F48B2F752F8E
:102BE0000DC06430710581F058F06630710579F4DC
:102BF0007E2F8B2F932F0DC0832F7B2F9E2F09C0ED
:102C00008E2F7B2F952F05C08E2F732F02C07E2F06
:102C1000852F692FDF91CF911F910F91FF90EF903A
:102C2000089541E00E948115089508950E941116AB
:102C30000895CF93DF93762FE901682F842F0E94A8
:102C40001616798368838A83DF91CF9108958091E6
:102C5000AB02282F269530E02115310519F481703B
:102C6000826005C02532310524F08170886480932C
:102C7000AB02089588E090E00C94C62BCF92DF92CF
:102C8000EF92FF926B017C010E942716B701A6010B
:102C900088E090E0FF90EF90DF90CF900C94E42BD1
:102CA000EBEAF2E083E0808311828FEF82838383FB
:102CB000148260817181828193810C943E1680918F
:102CC000AB0280FF02C08695089580E00895909140
:102CD000AF02933018F49F5F9093AF02882351F0B6
:102CE0006091AB027091AC028091AD029091AE0206
:102CF0000C943E16089581E00C9467169091AF02F3
:102D0000992319F091509093AF02882351F060916C
:102D1000AB027091AC028091AD029091AE020C9426
:102D20003E16089581E00C947E1670E00C94D61C3B
:102D3000609110018091AB0280FF0AC080910F0169
:102D400023E0829FC001112480559D4F0C9495165D
:102D50008091110190911201891780F7E82FF0E01E
:102D60009F01220F331FE20FF31FE055FD4F118229
:102D7000108212828F5FF0CF9091AB0290FF16C04D
:102D80009091110120911201921770F4E92FF0E057
:102D9000DF01AA0FBB1FEA0FFB1FE055FD4F818328
:102DA000608342839F5FF0CF0C9498160895CF9371
:102DB000DF9300D01F92CDB7DEB79091AB0290FFAA
:102DC0000AC09E012F5F3F4F0E9419164B816981F7
:102DD0008A810E94BC160F900F900F90DF91CF91C7
:102DE0000895CF93DF93EC016C8170E080E090E078
:102DF0000E940A2920E030E04FE753E40E942D288A
:102E00002BED3FE049E450E40E94332A0E94A02ABF
:102E10000E94A7282BE43AE34EE25FE30E94C0271A
:102E200020EF3BEF48ED52E40E94332A0E94D9285C
:102E3000462FEBEAF2E0628181810E94D7168C81F5
:102E40008F5F8C83DF91CF910895CF93DF93EC0157
:102E5000EBEAF2E0438162818C810E94D7168C817B
:102E60008F5F8C83DF91CF9108950F931F93CF9342
:102E7000DF9300D01F92CDB7DEB78C0180916E0238
:102E800081110AC09E012F5F3F4F4FEF6FEF0E94ED
:102E900019168A8180936E02F8018481813051F085
:102EA00028F0823061F440916E020AC080916E0277
:102EB00040E007C060916E0240E080E003C040E067
:102EC00080E060E00E94BC16F801848190E00196E9
:102ED00063E070E00E942B2B84830F900F900F9083
:102EE000DF91CF911F910F910895AF92BF92CF9232
:102EF000DF92EF92FF920F931F93CF93DF9300D057
:102F00001F92CDB7DEB7182FF62E042FE22E909128
:102F1000AB0290FF6DC0E92FE695AE2FB0E0AF5544
:102F2000BE4F8C9180937A029E7F923061F49E0115
:102F30002F5F3F4F812F0E9419164B8169818A8133
:102F40000E94BC1643C0823019F40091AE023EC00C
:102F5000863019F41091AC0239C08930D9F3893127
:102F6000A9F5E9518E2F8170D82EE695F0E0E85B47
:102F7000FD4FA590B490C12CBB2460911301C616DF
:102F800018F52C2D30E0A29EC001A39E900DB29E9C
:102F9000900D112470E00E94172B812FD11002C0D8
:102FA000860F01C0861B90911101290F311DA901C7
:102FB000440F551F240F351F20553D4F402F6F2DB7
:102FC0000E941916C394D9CF0E9498161093AC0290
:102FD000F092AD020093AE02EE2051F06091AB0290
:102FE0007091AC028091AD029091AE020E943E16AB
:102FF0000F900F900F90DF91CF911F910F91FF9045
:10300000EF90DF90CF90BF90AF900895EBEAF2E0A1
:103010009181282F4381628188E0890F0C94751774
:1030200081E00C940618EBEAF2E09181282F4381AD
:10303000628188EF890F0C94751781E00C94131846
:10304000EBEAF2E0628128E0620F08F46FEF282FCC
:10305000438181810C94751781E00C942018EBEA70
:10306000F2E0628128E0621B08F460E0282F4381CF
:1030700081810C94751781E00C942F18EBEAF2E033
:10308000438128E0420F08F44FEF282F62818181AD
:103090000C94751781E00C943E18EBEAF2E0438142
:1030A00028E0421B08F440E0282F628181810C94C3
:1030B000751781E00C944D1820E00C947517FF9261
:1030C0000F931F93CF93DF93EC01F12C0FEF10E0E0
:1030D00060911301F616F0F4809111012F2D30E06C
:1030E000280F311DC901880F991F280F391F20553E
:1030F0003D4F70E0C8010E942B2B962F8C81409190
:10310000AE026091AD02F99E800D11240E94191645
:10311000F394DECF0E9498169A818C8190FF02C0B2
:103120008F5F01C081508C83DF91CF911F910F91F0
:10313000FF900895AF92BF92CF92DF92EF92FF92ED
:103140000F931F93CF93DF93FC01828180FF02C016
:103150000FEF01C001E010E04CE0A42E80911301BC
:10316000181708F043C080911101C12ED12CE6013F
:10317000C80FD11DCE01880F991FC80FD91FC05588
:10318000DD4F198218821A8234E0E32EF12CB12C23
:10319000809170028B0D8D302CF06A2D0E94092BCE
:1031A000892F05C087FF03C090911301890F082E56
:1031B000000C990BC816D90691F48091AE028E9D31
:1031C000A0018F9D500D1124559547955595479514
:1031D0009E016091AD028091AC020E941916B00E62
:1031E000F1E0EF1AF108A1F61F5FB8CF0E94981620
:1031F00080917002013031F4811102C0809113017D
:10320000815007C090E001966091130170E00E9428
:103210002B2B80937002DF91CF911F910F91FF9024
:10322000EF90DF90CF90BF90AF900895CF938091B3
:10323000110190911201891770F4E82FF0E09F01BD
:10324000220F331FE20FF31FE055FD4F1182108252
:1032500012828F5FF0CFC0E060911301C617C0F5F6
:10326000EC2FF0E070E0CF010E942B2B2091110198
:10327000820F20916F02022E000C330B90E0E217B8
:10328000F307CCF020910E01022E000C330B2E1709
:103290003F078CF09C01220F331F820F931F9C016C
:1032A00020553D4F4091AE026091AD028091AC023D
:1032B0000E9419160BC0FC01EE0FFF1F8E0F9F1FFF
:1032C000FC01E055FD4F118210821282CF5FC4CF06
:1032D0000E94981620910D0180916F02820F8093B9
:1032E0006F0290910E01920F90930E0119165CF4EB
:1032F000082E000C990B4091130150E041505109E8
:10330000841795071CF0219520930D01CF91089506
:103310008F929F92AF92BF92CF92DF92EF92FF92E5
:103320000F931F93CF93DF938C01FC014481C42F33
:10333000D0E09E01DE010E946F2B9B01AC010E9438
:10334000852B6B017C01E0E2F0E0EC1BFD0BA5E5B9
:10335000B0E09B01AC010E94852B4B015C019F01F9
:10336000DF010E94672B9B01AC010E94902B9B0107
:10337000AC012C0D3D1D4E1D5F1DC501B4010E9409
:103380003F2BC22FD22F2A3228F4F3E02F9F900137
:1033900011240DC025E530E02C1B3109C901880F2F
:1033A000991F280F391F37FF02C02F5F3F4F3595F8
:1033B0002795C22FC095F12C85E5E82EED1A809156
:1033C0001301F816C8F4F1FC02C08E2D01C08D2F38
:1033D000909111012F2D30E0290F311DA901440FCB
:1033E000551F240F351F20553D4F4C2F6091AD02C6
:1033F0000E941916F394E3CF0E949816F801848175
:10340000811102C091E003C0803219F49FEF9093C4
:103410000C0190910C01890FF8018483DF91CF9109
:103420001F910F91FF90EF90DF90CF90BF90AF90E2
:103430009F908F9008950F931F93CF93DF93EC018C
:1034400000E010E080911301282F30E002171307ED
:1034500024F5909111019801290F311DA901440F04
:10346000551F240F351F20553D4F869590E04C8108
:10347000081719071CF4442331F002C0411103C09E
:103480004091AE0201C040E06091AD028091AC027B
:103490000E9419160F5F1F4FD5CF0E9498168C817E
:1034A00090E00196817099278C83DF91CF911F91D5
:1034B0000F910895EBEAF2E080818E7F8083608136
:1034C0007181828193810E943E1610927B022FEFC0
:1034D00080E792E0215080409040E1F700C000007A
:1034E0000C949816EBEAF2E080818E7F8083109234
:1034F0007B022FEF80E792E0215080409040E1F77F
:1035000000C000000C94981610927B028091780203
:1035100081110AC081E0809378028091AB028170B2
:10352000809377020C94721A08956091AB026695AD
:1035300070E04BE050E084E191E00E94A42B892BE5
:1035400019F481E080937B020E94832090937202A1
:103550008093710208959091AB0290FF35C09170F5
:10356000811102C0926006C0853210F0986402C0DA
:10357000880F982B9093AB02662351F06091AB02B9
:103580007091AC028091AD029091AE020E943E1605
:103590006091AB02669570E04BE050E084E191E011
:1035A0000E94A42B892B19F010927B0202C00E946A
:1035B000951A81E0809374024091AE026091AD0251
:1035C0008091AC020C945C180895682F9091AB0226
:1035D000969581E0890F853208F081E00C94AB1A52
:1035E00081E00C94E51A682F9091AB0296958FEFCD
:1035F000890F09F484E20C94AB1A81E00C94F31A5D
:1036000061E00C94AB1AEBEAF2E080818160808388
:1036100086950C94001B8091AB0280FD0C945A1A85
:103620000C94031B60E00C94AB1A80917902811119
:103630002EC00E94C20D811104C00E946A0E0E9419
:1036400050160E943A166093AB027093AC028093BE
:10365000AD029093AE026E7F61F40E9450160E94FC
:103660003A166093AB027093AC028093AD029093D4
:10367000AE020E94271610927B028091AB0280FF5F
:1036800003C086950E94121B81E080937902089501
:10369000EBEAF2E080818160808386950C94121BB6
:1036A000109278028091770281110E94481B0C943D
:1036B000951A0F931F93CF93DF9380917B028823FA
:1036C00009F485C080917A02E091AB02E695E81B8F
:1036D000E0937302823049F4F0E0EC5BFD4FE4913B
:1036E000CE2FD0E001EF16E149C0863049F4F0E07A
:1036F000EF5BFD4FE491CE2FD0E005E217E13EC035
:10370000893051F4E695F0E0E25CFD4FE491CE2F74
:10371000D0E00FE518E132C08F3051F4E695F0E0CB
:10372000E55CFD4FE491CE2FD0E00AE918E126C018
:10373000853149F4F0E0E85CFD4FE491CE2FD0E014
:1037400006E119E11BC0883181F0833239F4E6E3E8
:10375000F2E0C591D49105E317E110C0843251F431
:10376000C4EFD1E00BE11AE109C0C8E2D0E008E8FB
:1037700019E104C0C0EDD7E005E116E180917402C3
:10378000882361F0109274020E9483209093720249
:103790008093710210927602109275020E9483202B
:1037A000E0917102F09172028E1B9F0B8F3F9F4739
:1037B00070F4EC0FFD1FF0937202E093710281E749
:1037C00092E0F801DF91CF911F910F910994DF9161
:1037D000CF911F910F910895882311F0FA0101C034
:1037E000FB010994CF93DF93C82FD62F0E945F1659
:1037F0008C1740F00E945F168D1720F4DF91CF9157
:103800000C94F01A8C2FDF91CF910C94001B1F9316
:10381000CF93DF93FB0112811111C3C0EC010E9411
:10382000DF0C8272CD3CFCE5DF0709F49AC0A8F5F5
:10383000C73CECE5DE0709F476C0A8F4C43C9CE57F
:10384000D90709F45FC028F4C33CDC4509F457C02C
:1038500054C0C53C9CE5D90709F459C0C63CDC45B9
:1038600009F45CC04AC0CA3CFCE5DF0709F46AC041
:1038700050F4C83CECE5DE0709F45AC0C93CDC450D
:1038800009F45BC03AC0CB3C9CE5D90709F45FC0A2
:10389000CC3CDC4509F460C030C0C23DFCE5DF072C
:1038A00009F46FC088F4CF3C9CE5D90709F460C0E7
:1038B00008F45CC0C03DFCE5DF0709F45CC0C13D15
:1038C000DC4509F45BC019C0C53D9CE5D90709F486
:1038D00060C050F4C33DFCE5DF0709F455C0C43DAA
:1038E000DC4509F454C009C0C63D9CE5D90709F47C
:1038F00055C0CE35DD4509F454C011E052C00E94D8
:103900000B1B4FC04DEF5AE160EF7AE104C040EF6E
:103910005AE16DEF7AE10E94EC1B43C04DE158E1A2
:1039200060E178E1F8CF40E158E16DE178E1F3CF73
:103930004BE358E16CE278E1EECF4CE258E16BE307
:1039400078E1E9CF49E558E16AE478E1E4CF4AE477
:1039500058E169E578E1DFCF42E956E16BE776E1CE
:10396000DACF4BE756E162E976E1D5CF81E017C0C7
:1039700065E082E010C068E086E00DC06EE089E09E
:103980000AC064E18FE007C067E185E104C088E117
:1039900006C062E289E10E94F21B03C083E20E943A
:1039A000001B812FDF91CF911F910895259A25B19A
:1039B0002F7D35B130624FB7F894FC01CB01880FF1
:1039C000991F680F791F6E0F7F1FE617F70789F0A1
:1039D000819198E035B9000000C087FF25B9880FB4
:1039E000000000C000C000C025B900C09A9591F742
:1039F000ECCF4FBF8FE594E00197F1F700C00000D6
:103A00000895CF93DF93EC01FB018281882309F4B1
:103A10003CC1C430FDE5DF0760F4CB3F9CE5D9072E
:103A200088F49E0122503C452431310508F02EC116
:103A300009C0C236EDE5DE0729F0C63AFDE5DF072D
:103A400009F024C10E94D50D9093960280939502AF
:103A5000C1318CE5D80709F4C6C008F042C0C930AE
:103A6000ECE5DE0709F49BC000F5C5308CE5D8070E
:103A700009F485C078F4C330ECE5DE0709F478C0BA
:103A800008F07AC0C230DC4509F0F5C0809195029B
:103A90008160EFC0C7309CE5D90709F478C008F011
:103AA0007AC0809195028061E4C0CD30FCE5DF07EB
:103AB00009F487C058F4CB309CE5D90709F479C0E4
:103AC00008F07BC08091950288606FC0CF30FCE524
:103AD000DF0709F480C008F082C080919502877FDB
:103AE000C8C0CE3F9CE5D90709F471C000F5C531C7
:103AF000FCE5DF0709F485C068F4C3319CE5D9070C
:103B000009F475C008F095C00E948C078091950259
:103B10008F77AFC0CC3FFCE5DF07A9F108F054C0B8
:103B2000CB3FDC4509F0A7C08091960240C0C2306F
:103B3000EDE5DE0709F489C058F4C1158DE5D80715
:103B400009F45AC008F069C08091960282602FC0C3
:103B5000C236EDE5DE0709F47CC0C63AFDE5DF07B5
:103B600009F481C0C330DD4509F085C080E06EC036
:103B70008091950282607DC08091950216C08091EF
:103B80009502886076C08091960282604FC08091D5
:103B9000950280626EC08091950280646AC00E9426
:103BA0008C0780919502806864C0846062C08160E7
:103BB0003DC0809195028E7F5CC0809195028D7F83
:103BC00058C08091950216C08091960218C08091CD
:103BD00096028D7F2BC0809195028F7E4AC0809186
:103BE00095028F7D46C0809195028F7B42C0809167
:103BF0009502877F8B7F3DC0809196028D7F8E7F5F
:103C000015C08091950282FB222720F991E092272E
:103C100090FB82F990FB83F92CC080919602982F3B
:103C2000909591708E7F892B90FB81F980939602FD
:103C300022C00E948C078091950287FB222720F9E1
:103C400091E0922790FB87F914C081E00E946C0EEE
:103C500012C08091950284FB222720F991E09227DF
:103C600090FB84F906C080919502982F909590FB67
:103C700080F98093950280919502909196020E941E
:103C8000E60D0E948C0780E001C081E0DF91CF91BA
:103C90000895CF93DF9386319C4541F5EB010E9457
:103CA000DF0C982F8A812091020130910301882333
:103CB00079F09A7A81E009F480E080937C02911196
:103CC00002C069E201C065E3C9010E94DC1F0AC0AD
:103CD00080917C02811102C069E201C065E3C901E3
:103CE0000E94DE1F0E94210D80E001C081E0DF9173
:103CF000CF9108950F931F93CF93DF93C42FD22FAB
:103D0000FC0182818823C9F040937F020E948320B6
:103D100090937E0280937D0280E28C0F883008F0C1
:103D200057C0C77081E001C0880FCA95EAF7DF91DC
:103D3000CF911F910F910C94E90480917F02481359
:103D400030C080917D0290917E020E949B20883C31
:103D5000910538F510E21D0FCD17B9F080E28C0FF8
:103D6000883040F4C77081E001C0880FCA95EAF737
:103D70000E94F004183028F581E09D2F977001C053
:103D8000880F9A95EAF70E94E904802F0E94E004C8
:103D90001830F0F4D77081E001C0880FDA95EAF7A7
:103DA0000AC080E28C0F883098F4C77081E001C0AF
:103DB000880FCA95EAF7DF91CF911F910F910C946C
:103DC000F004802FDF91CF911F910F910C94E004AC
:103DD000DF91CF911F910F9108950F939C01CB011B
:103DE000243F4CE5340731F188F4293DFCE53F07D9
:103DF000D9F02A3D4CE5340779F1283D3C45A9F539
:103E000006E221EE41EE68ED7CE52BC0263FFCE5A5
:103E10003F07E1F0A8F0273F3C4539F507E225EEE2
:103E200046EE67EF7CE51DC007E225EE45EE69ED45
:103E30007CE517C006E221EE40EE64EF7CE511C0A0
:103E400007E225EE44EE65EF7CE50BC006E221EECD
:103E500042EE66EF7CE505C008E221E045EE6AED42
:103E60007CE50E947A1E80E008C0FC0182818823E4
:103E700019F010927F0201C081E00F910895909394
:103E8000C7018093C60108959093850280938402B0
:103E90000895E0918402F0918502309721F001901D
:103EA000F081E02D099480E00895E0918402F09182
:103EB0008502309721F00280F381E02D0994089566
:103EC000E0918402F0918502309739F022E0DC0124
:103ED0002C930480F581E02D0994089520918202AD
:103EE000309183022817390771F0909383028093F1
:103EF0008202E0918402F0918502309721F00680E1
:103F0000F781E02D0994089520918002309181027B
:103F10002817390771F09093810280938002E09115
:103F20008402F0918502309721F00084F185E02D24
:103F300009940895FC01329697E080E0915029F0B1
:103F400021912223D9F38F5FF9CF0895662349F099
:103F5000FC01329608962191621729F0E817F907BB
:103F6000D1F780E0089581E008959C01FC0132962C
:103F70009FEF80E04191461789F09F3F19F441116E
:103F800001C0982F8F5F8630A9F79F3F39F0F90164
:103F9000E90FF11D97FDFA956283089508959C013C
:103FA0002A5F3F4FFC014281461301C012820196F5
:103FB00082179307B9F708950C94B51F0C94CF1F7F
:103FC000029626E0FC0111922A95E9F708950895DA
:103FD0000C94E71F83E0809386020C94E81F811104
:103FE00002C081E001C082E0809386020C94E81F49
:103FF0000C94EF1F81E0809386020C94E81F0C94D0
:10400000FA1F08950C9401200C9402200C940120B6
:104010000C9401200C940120CF930E9408200E9450
:1040200059120E940620C0E08C2F0E948311892B18
:1040300029F4CF5FC530C1F780E001C081E0CF91A6
:10404000089508951F920F920FB60F9211248F9327
:104050009F93AF93BF9380918702811113C080918A
:10406000D4029091D502A091D602B091D702419688
:10407000A11DB11D8093D4029093D502A093D602C6
:10408000B093D702BF91AF919F918F910F900FBEC8
:104090000F901F9018958091DC02843031F10E94BE
:1040A00038031092870220E488E190E00FB6F8947C
:1040B000A895809360000FBE2093600083B7817F36
:1040C000846083BF83B7816083BF7894889583B70A
:1040D0008E7F83BF0FB6F894A895809160008861A9
:1040E00080936000109260000FBE08950E948C07BC
:1040F0000C943E0382E084BD93E095BD9AEF97BD9A
:1041000080936E0008952FB7F8948091D402909117
:10411000D502A091D602B091D7022FBF08952FB734
:10412000F8946091D4027091D5028091D60290915A
:10413000D7022FBF08959C014FB7F8948091D40205
:104140009091D502A091D602B091D7024FBF821BA9
:10415000930B089578941F920F920FB60F9211242B
:104160008F939F93AF93BF938091D4029091D50288
:10417000A091D602B091D7020196A11DB11D8093E6
:10418000D4029093D502A093D602B093D702BF91E8
:10419000AF919F918F910F900FBE0F901F90189528
:1041A00081E08093E00080E28093D8001092C90003
:1041B0008FE19EE40197F1F700C0000087E090EBEB
:1041C000DC018093E5029093E602A093E702B093AE
:1041D000E8029CE088E10FB6F894A895809360000F
:1041E0000FBE90936000FFCF8091930208950895D1
:1041F00022E02093E9002FEF3091E800215035FDB7
:1042000006C035ED3A95F1F700002111F5CF209168
:10421000E80025FF0BC040E050E066E070E00E943F
:1042200022238091E8008E778093E8000895CF9351
:10423000DF9321E02093E9002FEF3091E800215037
:1042400035FD06C035ED3A95F1F700002111F5CFA7
:104250002091E80025FF14C0EC0140E050E068E048
:1042600070E00E9422238091E8008E778093E8001E
:1042700088E0FE01ABE8B2E001900D928A95E1F78B
:10428000DF91CF9108958093880270938A026093A2
:1042900089028091DC02843001F582E08093E9009C
:1042A0008FEF9091E800815095FD06C095ED9A95AD
:1042B000F1F700008111F5CF8091E80085FF0DC076
:1042C00040E050E063E070E088E892E00E94222342
:1042D0008091E8008E778093E8000895BC0184E027
:1042E0000C944321BC0183E00C9443218091DB02B8
:1042F000811109C00E94B3240E9410258091E20020
:1043000084608093E20008951092DB0208950C947B
:10431000FF1F6091D80281E0611101C080E00C9420
:10432000EA1F9091DC0281E0943009F080E0609116
:10433000D8020C94EF1F42E061EC81E00E942C2433
:1043400042E261EC82E00E942C249091DC0281E048
:10435000943009F080E06091D8020C94F81F8091AD
:10436000DE02833009F461C030F4813071F08230B4
:1043700009F49AC008958A3009F486C08B3009F494
:104380006CC0893009F0A8C020C08091DD02813A5C
:1043900009F0A2C08091E800877F8093E8008091B7
:1043A000E1029091E202892B21F468E08BE892E02F
:1043B00003C060E080E090E070E00E946D23809197
:1043C000E8008B778093E80008958091DD028132C8
:1043D00009F082C08091E1029091E202029708F018
:1043E0007BC08091E800877F8093E8008091E8009F
:1043F00082FD05C08091DC028111F8CF6DC0209153
:10440000F3008091F20090E0922B029731F48091BA
:10441000F100813011F0863021F48091F100809319
:1044200093028091E8008B7753C08091DD02813A3E
:1044300009F052C08091E1029091E202892B09F0CB
:104440004BC08091E800877F8093E8008091E8006E
:1044500080FFFCCF80912B0136C08091DD0281323C
:10446000D9F58091E1029091E202892BA9F5809122
:10447000E800877F8093E8000E9461248091DF023A
:1044800080932B010C948C078091DD02813221F501
:104490008091E800877F8093E8000E9461248091EA
:1044A000E0028093940208958091DD02813AA1F4A4
:1044B0008091E800877F8093E8008091E80080FF8A
:1044C000FCCF809194028093F1008091E8008E7778
:1044D0008093E8000C946124089584B7877F84BF9B
:1044E0000FB6F894A8958091600088618093600071
:1044F000109260000FBE90E080E80FB6F8948093B1
:104500006100909361000FBE0C94FA1F0E94B324C7
:104510000E941025E2EEF0E0808184608083789430
:104520000C94A5278FE191E00C94441F8091DC024C
:104530008530A9F48091DC02853079F40E944B200B
:104540008091DA028823B1F30E940C20882391F332
:104550000E940C230E948C07EDCF0C9476200895C6
:1045600008950C94B322292F332723303105C9F045
:1045700060F42130310581F02230310509F044C06A
:104580008BE390E025E733E043C021323105E1F0D1
:104590002232310549F138C082E190E020EB33E06E
:1045A00037C099278130910549F028F0029761F5CD
:1045B000EDE4F3E005C0E1E7F3E002C0EDE5F3E090
:1045C000849190E09F0124C06115710541F0613034
:1045D0007105D1F489E090E020EA33E019C089E068
:1045E00090E027E833E014C06115710541F06130B7
:1045F000710551F48BE790E022EC33E009C080E4D0
:1046000090E02DE334E004C080E090E020E030E072
:10461000FA0131832083089580E189BD82E189BD5B
:1046200009B400FEFDCF8091D8008F7D8093D80023
:104630008091E00082608093E0008091E00081FD45
:10464000FCCF0895CF92DF92EF92FF920F931F93CA
:10465000CF93DF93EC018B017A010E9480248111BA
:1046600033C0E114F10439F0F70180819181081B16
:10467000190BC80FD91FC12CD12C0115110519F127
:104680008091E80085FD16C08091E8008E778093C8
:10469000E800E114F10449F0F70180819181C80E2E
:1046A000D91ED182C08285E00FC00E948024882359
:1046B00021F30AC089918093F10001501109FFEFA5
:1046C000CF1ADF0ADACF80E0DF91CF911F910F91EF
:1046D000FF90EF90DF90CF9008952091E30230910A
:1046E000E4022617370748F06115710539F4209167
:1046F000E8002E772093E80001C0B901FC0120E01A
:104700006115710579F18091DC028823F1F1853022
:10471000F1F18091E80083FD3CC08091E80082FDCA
:104720002EC08091E80080FFEBCF2091F3008091B4
:10473000F20090E0922B6115710551F088309105DF
:1047400038F421912093F100615071090196F3CF63
:1047500021E0089709F020E08091E8008E778093AF
:10476000E800CECF2111CFCF0AC08091DC02882390
:1047700061F0853061F08091E80083FD0AC080918E
:10478000E80082FFF2CF80E0089582E0089583E0A0
:10479000089581E008952091E3023091E402261704
:1047A000370748F06115710539F42091E8002E773C
:1047B0002093E80001C0B901FC0120E061157105FA
:1047C00091F18091DC02882309F440C0853009F41E
:1047D0003FC08091E80083FD3DC08091E80082FDEC
:1047E0002FC08091E80080FFE9CF2091F3008091F5
:1047F000F20090E0922B6115710559F08830910517
:1048000040F424912093F100319661507109019692
:10481000F2CF21E0089709F020E08091E8008E7740
:104820008093E800CBCF2111CCCF0AC08091DC026D
:10483000882361F0853061F08091E80083FD0AC033
:104840008091E80082FFF2CF80E0089582E0089531
:1048500083E0089581E00895982F973068F590934C
:10486000E900981739F07091EC002091ED0050911B
:10487000F00003C0242F762F50E021FD02C09F5F7F
:10488000ECCF3091EB003E7F3093EB003091ED00A8
:104890003D7F3093ED003091EB0031603093EB00C1
:1048A0007093EC002093ED005093F0002091EE0007
:1048B00027FDE5CF80E008958F708093E90081E0C7
:1048C00008958091DD0287FF11C08091E80082FD8C
:1048D00005C08091DC028111F8CF11C08091E80001
:1048E0008B770BC08091DC02882349F08091E8002F
:1048F00080FFF8CF8091E8008E778093E8000895DC
:104900002091E4003091E50095E64091EC00842F81
:10491000817040FF23C08091E80080FD1DC0809120
:10492000DC02882399F0853099F08091EB0085FDB9
:1049300011C04091E4005091E5002417350729F398
:10494000915011F09A01E1CF84E0089582E008953A
:1049500083E0089581E0089580E008954091E800A3
:1049600042FFDDCF08950E9421250E942925E0EE17
:10497000F0E0808181608083E8EDF0E080818F77D6
:10498000808319BCA7EDB0E08C918E7F8C938081E1
:104990008F7E80831092DB0208950F931F93CF9335
:1049A000DF930E9421250E942925C8EDD0E088814F
:1049B0008F77888388818068888388818F7D8883CA
:1049C00019BC1092DC021092D8021092DA021092F6
:1049D000D90200EE10E0F80180818B7F808388810E
:1049E0008160888342E060E080E00E942C24E1EE58
:1049F000F0E080818E7F8083E2EEF0E08081816054
:104A00008083808188608083F80180818E7F8083AD
:104A1000888180618883DF91CF911F910F910895E4
:104A2000E8EDF0E080818F7E8083E7EDF0E080812B
:104A30008160808384E082BF81E08093DB020C94FC
:104A4000CD24E8EDF0E080818E7F80831092E2003B
:104A500008951092DA001092E10008951F920F92CB
:104A60000FB60F9211242F933F934F935F936F9341
:104A70007F938F939F93AF93BF93EF93FF93809117
:104A8000E10082FF0BC08091E20082FF07C08091AD
:104A9000E1008B7F8093E1000E94A4278091DA00DF
:104AA00080FF1FC08091D80080FF1BC08091DA007A
:104AB0008E7F8093DA008091D90080FF0DC080E165
:104AC00089BD82E189BD09B400FEFDCF81E08093FC
:104AD000DC020E94762105C019BC1092DC020E9403
:104AE00084218091E10080FF19C08091E20080FF65
:104AF00015C08091E2008E7F8093E2008091E200F9
:104B000080618093E2008091D80080628093D80019
:104B100019BC85E08093DC020E9489218091E1002C
:104B200084FF30C08091E20084FF2CC080E189BD09
:104B300082E189BD09B400FEFDCF8091D8008F7D50
:104B40008093D8008091E1008F7E8093E100809176
:104B5000E2008F7E8093E2008091E200816080938A
:104B6000E2008091D802882311F084E007C0809190
:104B7000E30087FD02C081E001C083E08093DC0296
:104B80000E9491218091E10083FF29C08091E20081
:104B900083FF25C08091E100877F8093E10082E060
:104BA0008093DC021092D8028091E1008E7F809386
:104BB000E1008091E2008E7F8093E2008091E2002C
:104BC00080618093E20042E060E080E00E942C245B
:104BD0008091F00088608093F0000E948721FF910F
:104BE000EF91BF91AF919F918F917F916F915F9165
:104BF0004F913F912F910F900FBE0F901F901895DE
:104C00001F920F920FB60F9211242F933F934F9341
:104C10005F936F937F938F939F93AF93BF93CF9344
:104C2000DF93EF93FF93C091E900CF708091EC0088
:104C3000D82FD17080FDD0E81092E9008091F0006B
:104C4000877F8093F00078940E9444261092E900B8
:104C50008091F00088608093F000CD2BCF70C093DE
:104C6000E900FF91EF91DF91CF91BF91AF919F91BB
:104C70008F917F916F915F914F913F912F910F9005
:104C80000FBE0F901F9018951F93CF93DF93CDB752
:104C9000DEB7AA970FB6F894DEBF0FBECDBFEDED1D
:104CA000F2E08091F100819322E0E53EF207C9F73E
:104CB0000E94AF218091E80083FF2EC18091DD0228
:104CC0009091DE02492F50E04A30510508F024C18E
:104CD000FA01EE59FF4F0C94612B803821F0823895
:104CE00009F01AC108C08091D9029091DA02992383
:104CF00089F082600FC08091E1028F70873008F0E8
:104D00000BC18093E9008091EB0085FB882780F937
:104D10001092E9009091E800977F9093E8008093CB
:104D2000F1001092F100D1C0282F2D7F09F0F4C0BE
:104D3000882319F0823061F0EFC08091DF0281306A
:104D400009F0EAC0933009F080E08093DA022EC0C7
:104D50008091DF0281112AC08091E1028F702FEFD4
:104D6000280F263008F0D8C08093E9002091EB008E
:104D700020FF1CC0933021F48091EB00806214C0AE
:104D80009091EB0090619093EB0021E030E0A9015D
:104D900002C0440F551F8A95E2F74093EA00109233
:104DA000EA008091EB0088608093EB001092E900AC
:104DB0008091E800877F8093E8000E946124ACC066
:104DC0008111AAC01091DF021F778091E3008078E3
:104DD000812B8093E3008091E800877F8093E80037
:104DE0000E9461248091E80080FFFCCF8091E30065
:104DF00080688093E300111102C082E001C083E06B
:104E00008093DC0289C08058823008F085C0809190
:104E1000DF029091E0028C3D53E0950779F583E045
:104E20008A838AE289834FB7F894DE01139620E0E3
:104E30003EE051E2E32FF0E050935700E49120FF71
:104E400003C0E295EF703F5FEF708E2F90E0EA3085
:104E500010F0C79601C0C0968D939D932F5F2431AB
:104E600049F74FBF8091E800877F8093E8006AE2AE
:104E700070E0CE0101960E946D2316C06091E102A0
:104E80007091E202AE014F5F5F4F0E94B122BC0100
:104E9000892B09F441C09091E800977F9093E80036
:104EA00089819A810E94CB238091E8008B7780933F
:104EB000E80032C0803881F58091E800877F8093D8
:104EC000E8008091D8028093F1008091E8008E770D
:104ED00072CF811121C08091DF029091E002992769
:104EE0000297D4F48091E800877F8093E800809156
:104EF000DF028093D8020E9461248091D802811140
:104F000006C08091E30087FD02C081E001C084E01B
:104F10008093DC020E949B218091E80083FF0AC0FD
:104F20008091E800877F8093E8008091EB008062A9
:104F30008093EB00AA960FB6F894DEBF0FBECDBFEC
:104F4000DF91CF911F9108950895CF938091DC0256
:104F50008823A1F0C091E900CF709091EC00892FD7
:104F6000817090FD80E8C82B1092E9008091E800E4
:104F700083FD0E944426CF70C093E900CF9108952D
:104F80005058BB27AA270E94D8270C9483290E9437
:104F9000752938F00E947C2920F039F49F3F19F4DC
:104FA00026F40C944B290EF4E095E7FB0C9445296C
:104FB000E92F0E94942958F3BA17620773078407F0
:104FC000950720F079F4A6F50C94B6290EF4E09537
:104FD0000B2EBA2FA02D0B01B90190010C01CA01B3
:104FE000A0011124FF27591B99F0593F50F4503E5E
:104FF00068F11A16F040A22F232F342F4427585F50
:10500000F3CF469537952795A795F0405395C9F767
:105010007EF41F16BA0B620B730B840BBAF091501F
:10502000A1F0FF0FBB1F661F771F881FC2F70EC0BE
:10503000BA0F621F731F841F48F487957795679591
:10504000B795F7959E3F08F0B0CF9395880F08F07D
:105050009927EE0F9795879508950E9441280C9403
:1050600083290E947C2958F00E94752940F029F478
:105070005F3F29F00C94452951110C94B7290C94E9
:105080004B290E94942968F39923B1F3552391F396
:10509000951B550BBB27AA2762177307840738F0A7
:1050A0009F5F5F4F220F331F441FAA1FA9F335D004
:1050B0000E2E3AF0E0E832D091505040E695001CB8
:1050C000CAF72BD0FE2F29D0660F771F881FBB1F72
:1050D000261737074807AB07B0E809F0BB0B802D50
:1050E000BF01FF2793585F4F3AF09E3F510578F07C
:1050F0000C9445290C94B7295F3FE4F3983ED4F310
:10510000869577956795B795F7959F5FC9F7880F4F
:10511000911D9695879597F90895E1E0660F771FA1
:10512000881FBB1F621773078407BA0720F0621B32
:10513000730B840BBA0BEE1F88F7E095089529F4E2
:1051400016F00C9445290C94B6290C944B290E9416
:105150009C29A8F39638A0F707F80F92E8942BE360
:105160003AEA48EB5FE70E94492A0F920F920F92AA
:105170004DB75EB70F920E94FF29E8EDF0E00E9464
:105180004E294F915F91EF91FF91E595EE1FFF1F23
:1051900049F0FE57E0684427EE0F441FFA95E1F707
:1051A0004195550B0E94C9290F9007FE0C94BD290B
:1051B00008950E949C2988F09F5798F0B92F99274D
:1051C000B751B0F0E1F0660F771F881F991F1AF0F2
:1051D000BA95C9F714C0B13091F00E94B629B1E078
:1051E00008950C94B629672F782F8827B85F39F077
:1051F000B93FCCF3869577956795B395D9F73EF48B
:1052000090958095709561957F4F8F4F9F4F089532
:10521000E89409C097FB3EF4909580957095619550
:105220007F4F8F4F9F4F9923A9F0F92F96E9BB2706
:105230009395F695879577956795B795F111F8CF82
:10524000FAF4BB0F11F460FF1BC06F5F7F4F8F4FED
:105250009F4F16C0882311F096E911C0772321F0E3
:105260009EE8872F762F05C0662371F096E8862F7B
:1052700070E060E02AF09A95660F771F881FDAF7D2
:10528000880F9695879597F9089597F99F6780E815
:1052900070E060E008959FEF80EC0895DF93CF9376
:1052A0001F930F93FF92EF92DF927B018C01689422
:1052B00006C0DA2EEF010E94462AFE01E894A5916D
:1052C0002591359145915591A6F3EF010E94D8277C
:1052D000FE019701A801DA9469F7DF90EF90FF9043
:1052E0000F911F91CF91DF91089500240A94161613
:1052F000170618060906089500240A9412161306C4
:10530000140605060895092E0394000C11F4882351
:1053100052F0BB0F40F4BF2B11F460FF04C06F5F6D
:105320007F4F8F4F9F4F089557FD9058440F551F43
:1053300059F05F3F71F04795880F97FB991F61F017
:105340009F3F79F087950895121613061406551F8E
:10535000F2CF4695F1DF08C0161617061806991FFA
:10536000F1CF86957105610508940895E894BB27EF
:1053700066277727CB0197F908959B01AC0160E080
:1053800070E080E89FE30C942D280C9445290C9440
:10539000A82A0E949C29D8F39923C9F3940F511D80
:1053A000A3F39150504094F059F0882332F0660FE7
:1053B000771F881F91505040C1F79E3F51052CF731
:1053C000880F911D9695879597F908955F3FACF0EA
:1053D000983E9CF0BB27869577956795B79508F41E
:1053E000B1609395C1F7BB0F58F711F460FFE8CF98
:1053F0006F5F7F4F8F4F9F4FE3CF0C94B729FA0118
:10540000DC01AA0FBB1F9B01AC01BF5728F4222768
:1054100033274427507820C0B75190F4AB2F002495
:10542000469537952795011CA395D2F3002071F07E
:10543000220F331F441FB395DAF30ED00C94C0270C
:1054400061307105A0E88A07B94630F49B01AC01D0
:105450006627772788279078309621F0208331833C
:105460004283538308950E94462A0C9483290E9404
:10547000752938F00E947C2920F0952311F00C94B6
:1054800045290C944B2911240C94B7290E94942986
:1054900070F3959FC1F3950F50E0551F629FF00187
:1054A000729FBB27F00DB11D639FAA27F00DB11DA0
:1054B000AA1F649F6627B00DA11D661F829F222729
:1054C000B00DA11D621F739FB00DA11D621F839FB0
:1054D000A00D611D221F749F3327A00D611D231F86
:1054E000849F600D211D822F762F6A2F11249F57D4
:1054F00050409AF0F1F088234AF0EE0FFF1FBB1FD7
:10550000661F771F881F91505040A9F79E3F510595
:1055100080F00C9445290C94B7295F3FE4F3983E42
:10552000D4F3869577956795B795F795E7959F5F3F
:10553000C1F7FE2B880F911D9695879597F90895D1
:105540009F930E94B82A0F9007FCEE5F0C94E12A0B
:105550009F3F31F0915020F4879577956795B795E7
:10556000880F911D9695879597F908950C944B296E
:105570000E949C29D8F3E894E0E0BB279F57F0F005
:105580002AED3FE049EC06C0EE0FBB0F661F771F08
:10559000881F28F0B23A62077307840728F0B25ACE
:1055A000620B730B840BE3959A9572F7803830F495
:1055B0009A95BB0F661F771F881FD2F790480C94EF
:1055C000AA2AEF93E0FF07C0A2EA2AED3FE049ECE8
:1055D0005FEB0E94D8270E9483290F90039401FC5F
:1055E0009058E0E0F1E00C94F52A9F938F937F931D
:1055F0006F93FF93EF939B01AC010E94332AEF91CD
:10560000FF910E944E292F913F914F915F910C94F1
:10561000332A87FB082E062687FD819567FD619555
:105620000E94982B0EF4919507FC81950895AA1B72
:10563000BB1B51E107C0AA1FBB1FA617B70710F07D
:10564000A61BB70B881F991F5A95A9F780959095AF
:10565000BC01CD01089597FB072E16F4009407D0E6
:1056600077FD09D00E94172B07FC05D03EF49095DA
:1056700081959F4F0895709561957F4F0895A1E2A0
:105680001A2EAA1BBB1BFD010DC0AA1FBB1FEE1FBC
:10569000FF1FA217B307E407F50720F0A21BB30B07
:1056A000E40BF50B661F771F881F991F1A9469F783
:1056B00060957095809590959B01AC01BD01CF01DF
:1056C0000895EE0FFF1F0590F491E02D09940E94BC
:1056D0006F2B332312F48A1B9B0B0C94802BA29FFD
:1056E000B001B39FC001A39F700D811D1124911DB6
:1056F000B29F700D811D1124911D08950E946F2B82
:10570000B7FF0895821B930B08950E946F2BA59FEE
:10571000900DB49F900DA49F800D911D11240895AC
:10572000B7FF0C94852B0E94852B821B930B089549
:10573000991B79E004C0991F961708F0961B881FE3
:105740007A95C9F780950895FC014150504030F09A
:1057500001900616D1F73197CF0108958827992730
:105760000895FB01DC0104C08D910190801921F4A2
:1057700041505040C8F7881B990B0895F999FECF06
:1057800092BD81BDF89A992780B50895A6E1B0E051
:1057900044E050E00C94F82BA8E1B0E042E050E087
:1057A0000C94F82B262FF999FECF92BD81BDF89A63
:1057B000019700B4021639F01FBA20BD0FB6F89455
:1057C000FA9AF99A0FBE08950396272F0E94D32BB9
:1057D0000E94D22B252F0E94D32B242F0C94D32B45
:1057E0000196272F0E94D32B0C94D22BDC01CB01E6
:1057F000FC01F999FECF06C0F2BDE1BDF89A3196E1
:1058000000B40D9241505040B8F70895F894FFCF7E
:10581000C8004102280850011E0A140101010200BB
:105820000C000C0C01191A1B1C1D1E1F202122F438
:10583000201721F82072216E21F72001E200E900F3
:10584000EA00B500B600B700CD008301CC008A01A4
:10585000920194012102230224022502260227023A
:105860002A02B300B4006F007000818283E200E975
:1058700000EA00B500B600B700CD008301CC008A75
:10588000019201940121022302240225022602270B
:10589000022A02B300B4006F007000818283F4F525
:1058A000F6F731333632C69766949091F0F16795EA
:1058B0003700010202020206060609090909090960
:1058C0000F0F0F0F0F0F1515151819191919191991
:0658D00019191919232427
:00000001FF
